:060000001F308A000028F9
:1030000003138316203099000D2803138312A101A6
:1030100083168B138B1B052812288312A101A11480
:103020008316181518080439223898001F308A00B2
:1030300007178717D7308100831290309800C60198
:10304000C501A001C00140149526F1250526A01C4C
:103050002F28A11C2F2861233D21201D7C28A0178B
:103060008220A013201B3728A0187C282F282C266C
:10307000612361210008A821AC00031938285730CA
:103080002C02031D4528CF20382852302C02031D66
:103090004B28A5203828840A0008031D7A283F30D1
:1030A0002C02031D55287E25382855302C02031D7F
:1030B00066289522201D3828A01962285D25F62053
:1030C00005263828312189231E25382844302C0232
:1030D000031D6C28BE21382851302C02031D742892
:1030E000A0187C280526382856302C02031D7A2883
:1030F000052638289B243828A01C38284F261E3047
:103100008A00FC2E2013A328503092216130922196
:10311000733092219221773092216F309221723058
:103120009221643092213E30922161212208F627BB
:103130000002031DA42800080319A328A219A4282B
:10314000A20A840A962820170800840A2030000268
:10315000031DB628840AA0119921A800A019B62839
:103160000008031DB6282424B82008009B2408006A
:103170002808C420203092213D3092212030922115
:103180002708C42089230800B900F039B000300EA8
:10319000E527922139080F39E52792210800840A92
:1031A00020300002031DF428840AA0119921A019DF
:1031B000F428A70020300002031DF428840A4030C0
:1031C0000002031DF428840A20300002031DF428A5
:1031D000840A9921A800A019F4280008031DF428E6
:1031E00004242424B82008009B2408001F30A500D4
:1031F000C530A6003430A30049256121A20A000889
:10320000A4009523000803190800A60A840AA20A4C
:10321000A21A8001FF286400201018191329981C95
:103220001529181218161A0808008C1E08002014F8
:103230001A08C3000A3C0319201043080800810142
:103240000B110B21201C252908000B1D2129A11978
:103250000800C50A0319C60AC61E0800A0187C2863
:103260000800A1151F21201831291F2120183129FC
:103270001F2120183129A11108002011A1150F309C
:10328000BE000F30AB0020309221AB0B43293C3005
:1032900092211030AB0008309221AB0B4B290F303C
:1032A000AB001F2120185D29BE0B51290F30BE0035
:1032B00023309221AB0B51295E292015A1118923BE
:1032C000080050308400C601C5011F21201C65295B
:1032D00008304302031D7B2950300402031963297F
:1032E00084030830211C92212030211C92210830B7
:1032F000211C922163290D30430203198B294308B5
:103300008000A01B2A30211C92217F300402031967
:103310008B29840A6329211C89238001A201503052
:103320008400080081010B1164000C1E942999008F
:1033300008000008A8217D26A0190800B000B00EE2
:10334000840A0008A8217D26B0043008840A0800F9
:10335000C3007B3043020318B42961304302031CCD
:10336000B42920304302080043080800EE233F3010
:103370002302031D0800FF3024020800A0110526C7
:10338000A01C0800A501A601B101B621031DCF298B
:10339000A60A0319A50A3024A01DC429EA29250874
:1033A000BA002608BB00B10A2608AF00A60A031916
:1033B000A50A2F082606F839031DE4293024A01990
:1033C000E929B621031DD32923223024A019EA2993
:1033D000C4292322FA21A0113A3092210030C420BE
:1033E0000030C4200030C4200130C420FF30C4208D
:1033F00089230800A8014230BF003A3092211030E2
:10340000B200B6000310B60CC4200310280D031838
:103410003F143F08B207C4200310280DB207C42090
:103420000301C42024242708B207C4200301C420B8
:10343000A80AB60B122AB209320AC4208923280826
:10344000031DFD2908003A08A5003B08A6003A30F4
:1034500092210310310DB200C420260D250DB207B4
:10346000C4200310260DB207C4200301C420EE239C
:10347000A60A0319A50A2408B207C4202308B20724
:10348000C420B10B372AB209320AC42089230800AC
:103490004530922172309221613092217330922115
:1034A000693092216E309221673092218923A010D9
:1034B000A5010330A6003F30A300FF30A4009523F0
:1034C000A0190800A60A031D682AA50A2330922124
:1034D0003024A01D5F2AA0111F30A500C530A60012
:1034E0003430A300A4019523A0190800A60AE530F2
:1034F0002602031D732A1E30A500FC30A6003F30B3
:10350000A300FF30A4009523A0190800A60A031DFC
:10351000832AFF30A800FF30A7000424A019080068
:10352000A80B8D2A042489230800A0112011B301BF
:10353000B401B5014130922172309221653092215F
:1035400020309221793092216F3092217530922172
:103550002030922173309221753092217230922165
:10356000653092213F309221203092215B309221B0
:10357000793092212F3092214E3092215D3092216C
:103580003E30922161210008A821593C031D08000A
:10359000840A0008031D080020154822A01908000D
:1035A0005230922165309221613092216430922113
:1035B0007930922189232116211461212110B30A27
:1035C0000A303302031CEC2AB301B40A0A30340275
:1035D000031CEC2AB401B50A00083A3C031D442B35
:1035E000840A9921A0190800B100B2000310310C1F
:1035F000B100B8009921A0190800A500B2079921CF
:10360000A0190800A600B2070310A50CA60C99216A
:10361000A0190800B700B207B708031D402B040823
:10362000C200B10803191E2B9921A0190800B20786
:103630009921A0190800B207B103112B9921A019F3
:103640000800B207031D572B42088400B808031D69
:103650002C2B23309221DC2A9921A4009921A3004C
:103660003024A0194124A0190800A01E9523A01AF7
:103670005B23A0190800A60A0319A50AB803262B84
:10368000892337030319472BA015D7240800992154
:10369000A0190800B207031D572BF125A018080038
:1036A000A0156A23B301B401B501B30A0800A0153F
:1036B0008923F12408002408A7002608A800042470
:1036C00008005030922149309221433092213E30FF
:1036D00092210800303092219221922132309221A1
:1036E0006830922120309221213092213D30922168
:1036F00020309221673092216F30922174309221D4
:103700006F309221203092215830922192218923CA
:1037100008000A3092210D309221080020309221B9
:103720002D30922120309221080020126400203098
:103730002502031908002508C7002608C800250827
:10374000031DAA2B033026020318AA2B1E30A50046
:10375000FC30A607250803178F000313260803175C
:103760008D000313230803178E0003132408031787
:103770008C0083168C170C1555308D00AA308D00E7
:103780008C14FF3FFF3FFF3FFF3FFF3FFF3FFF3FE7
:10379000FF3FFF3FFF3FFF3FFF3FFF3FFF3FFF3F39
:1037A000FF3F000000000C110C1400000000831209
:1037B0000E0803132302031DE32B03170C08031346
:1037C00024020319E92B201AE72B2016AA2B7E24AA
:1037D000A0154708A5004808A600080064002508B1
:1037E00003178F000313260803178D0083168C1709
:1037F0000C140000000083120E080313A30003172B
:103800000C080313A40008000D12280803178D00EC
:103810000313270803178C0083168C130C155530DF
:103820008D00AA308D008C148312031364000D1ECA
:10383000162C031783160C110C1483120C08031397
:103840002702031D8C2408006400280803178D003C
:1038500083168C130C1483120C080313A7000800A2
:10386000A01218302502031C08002508203C03196B
:1038700008002508213C031D3F2CA0160800A015B8
:1038800008004D309221653092216D3092216F30C9
:103890009221723092217930922120309221703021
:1038A0009221723092216F309221743092216530D2
:1038B00092216330922174309221693092216F30CD
:1038C00092216E3092210425122508002030922189
:1038D00070309221723092216F30922167309221A4
:1038E00072309221613092216D30922192216930A3
:1038F00092216E3092216730922108004630922149
:103900004C30922141309221533092214830922103
:10391000662404251225080045309221922150305A
:103920009221523092214F3092214D3092216624C3
:103930008923A0150800C624633092216F3092219C
:103940006D3092219221613092216E30922164304B
:103950009221892308004E3092216F3092216E30DF
:1039600092212D30922148309221453092215830B9
:10397000922120309221633092216830922161306F
:103980009221723092210425892308004930922126
:103990006E30922176309221613092216C309221EA
:1039A0006930922164309221203092210800C6248F
:1039B0007230922165309221633092216F309221D2
:1039C0007230922164309221203092217430922101
:1039D000793092217030922165309221042589231B
:1039E0000800433092216830922165309221633083
:1039F00092216B30922173309221753092216D307B
:103A000092210425892308002030922165309221DB
:103A10007230922192216F309221723092212030A7
:103A20009221080040309221203092212508C420A4
:103A30002608C42068309221892308004C30922146
:103A4000693092216E30922165309221203092218E
:103A50006E309221753092216D3092216230922128
:103A6000653092217230922120309221A0123508C7
:103A700003193D2DA016E52792213408A01A422DE6
:103A80000319442DE52792213308E5279221892344
:103A90000800453092216E309221743092216530B9
:103AA0009221723092212030922161309221203077
:103AB0009221BC253E309221080055309221703071
:103AC00092216C3092216F309221613092216430CA
:103AD00092212030922173309221753092216330EF
:103AE0009221922165309221733092216630922189
:103AF000753092216C30922189230800C001C014D6
:103B0000952666268923553092218E2355309221A1
:103B1000703092216C3092216F309221613092216D
:103B2000643092216626743092216F309221D12523
:103B3000443092218E23443092216F30922177308D
:103B400092216E3092216C3092216F30922161303F
:103B50009221643092216626663092217230922141
:103B60006F3092216D309221D125C00140159526EC
:103B70006626BC2589230800723092216530922187
:103B8000763092212030922173309221743092212C
:103B900072309221693092216E30922167309221E9
:103BA00008002030922170309221723092216F30C3
:103BB00092216730922172309221613092216D30D2
:103BC0009221203092216D309221653092216D300A
:103BD00092216F3092217230922179309221892383
:103BE0000800A0101E30A500FC30A600EE2323081C
:103BF0003839283A0319032EFE30A600EE23230895
:103C00003839283A0319A0140800A01C122EC52721
:103C1000FF390319242EC00140169526C001C01596
:103C200095262A2E4E3092216F30922166266C30D6
:103C300092216F309221613092216430922165305F
:103C40009221643092212A2E4E3092216F3092219F
:103C50006626BC258923080043263F309221203068
:103C60009221663092216F30922172309221203061
:103C7000922168309221653092216C30922170300F
:103C800092218923080050309221723092216530B0
:103C900092217330922192212030922108004A30E3
:103CA0009221753092216D309221703092216930CD
:103CB00092216E309221673092212030922174300F
:103CC00092216F30922166268923080020309221AC
:103CD0007530922173309221653092217230922199
:103CE00020309221633092216F30922164309221F2
:103CF00065309221203092210800AF003030AF02B1
:103D0000031C922E0A302F02031C902E1130AF029A
:103D1000031C922E06302F020318922E0A30AF0792
:103D20002F080800A015AB240034AF012F0840185D
:103D30008C27C0185F2740190027C019C427401AD4
:0E3D40004D27FF39031908009221AF0A962E75
:103E00008207573420342D342034573472346934C7
:103E100074346534203474346F342034453445347C
:103E2000503452344F344D342C34203422345734EF
:103E30002034443444342034403420344134413438
:103E400022340A340D34523420342D342034523488
:103E50006534613464342034663472346F346D34C4
:103E6000203445344534503452344F344D342C349E
:103E700020342234523420344134413422340A3440
:103E80000D34563420342D342034443469347334A2
:103E900070346C34613479340034820743347534BF
:103EA0007234723465346E347434203469346D3451
:103EB00061346734653420343D3420340034820763
:103EC0003F3420342D342034443469347334703416
:103ED0006C34613479342034743468346934733424
:103EE00020346C346934733474340A340D345134EE
:103EF00020342D34203451347534693474342034F2
:103F000061346E34643420346A3475346D34703402
:103F1000203474346F34003482071B345B34323401
:103F20004A3438344B3420345034493443344C34DC
:103F30004F344134443445345234203476343134AF
:103F40002E34333431340A340D34A93452342E34FF
:103F50004634613472346D34653472342F345234E3
:103F60002E345034653472346434723469346134BC
:103F70007534203431343934393439340A340D3419
:023F800000340B
:083F880082070034003400340C
:103F90000034003400340034003400340034003481
:103FA0000034003400340034003400340034003471
:103FB0000034003400340034003400340034003461
:103FC000003400340034003400348207303431349B
:103FD0003234333434343534363437343834393495
:103FE00041344234433444344534463482074834FF
:103FF00065346C346C346F343134323433340034DF
:02400E00723FFF
:00000001FF
